:03000000020016E5
:030003000200C137
:100013000200DBD288D28AD2AFC2A8C2AA75F0D9B5
:100023001200741201FD74AF12021074A5120210B3
:1000330075400F1201CC74A412021012011B7540FB
:100043000F1201CC7B001200F575400F1201CC7B1F
:10005300081200F575400F1201CC12018A75401E7B
:100063001201CC74AE12021075400F1201CC0200C3
:10007300291201BF1201BFC291001201BFD2910028
:100083001201BF74A212021074A012021074C812DB
:10009300021074251202107481120210E5F012028C
:1000A3001074F81202107400120210742F1202104E
:1000B3001201BF744012021074A612021022C0E093
:1000C300E5F0B4C0030200D814F5F07481120210F5
:1000D300E5F0120210D0E032C0E0E5F0B4FF030215
:1000E30000F204F5F07481120210E5F0120210D050
:1000F300E0327AB0EA120210741012021074001285
:10010300021079109002467808EB9312022BA3D8C1
:10011300F8D9F10ABAB8DD2274B0120210741012C1
:100123000210740012021074FF12022B74011201E8
:10013300B374FF12022B74B1FD1202107410120279
:100143001074001202107E0674FF12022B74001248
:1001530001B374FF12022B0DED1202107410120280
:10016300107400120210DEE074B712021074101241
:100173000210740012021074FF12022B7480120119
:10018300B374FF12022B2274B0FD7F047E0290022F
:100193005EED120210741012021074001202107B32
:1001A3008074009312022BA3DBF70DDEE4DFDD2264
:1001B3007F7EC0E012022BD0E0DFF722754032755C
:1001C3004130D541FDD540F722D2A8D2AA1201FD74
:1001D3007541FA75425020970A1201FD00003097CD
:1001E3000B80F9D542F0D541EAD540E4C2A8C2AAB2
:1001F3002279197A32DAFED9FA227543047544FA60
:100203007545C8D545FDD544F7D543F122C0E0C2B5
:1002130090C2920075490833929400C2930000D2B1
:1002230093D549F300D0E022C0E0C290D29200758A
:10023300490833929400C2930000D293D549F30046
:10024300D0E022FF00FF00FF00FF0055AA55AA558A
:10025300AA55AA00000000000000000404FCFC04EE
:100263000404040C18F0E0000404FCFC0404003053
:1002730078CCC48484083C00000404FCFC0404041B
:100283008CF870000404FCFC04040000000000006F
:10029300000000C0300C7CF08000000004040C1C43
:1002A30074E480008064140C041C0C040404FCFC3F
:1002B3000404040C1C0404FCFC848484E4041C0077
:1002C30000C0F018080404040408083C000404FCFB
:1002D300FC8484808484FCFC04040020203F3F20B1
:1002E30020202010180F070020203F3F2020003C33
:1002F3001810202121331F0E0020203F3F21210110
:100303000100000020203F3F2020202020300C202F
:1003130030382702020202233F3C30200000000055
:1003230020203F3F202000000000000020203F3F0E
:10033300202000000020203F3F20202023203008E1
:1003430000070F1830202020202010080020203F15
:100353003F20200020203F3F2020001010F0F0100D
:100363001010103060C080001010F0F0101000C0AA
:10037300E03010101020F000001010F0F0101010FA
:1003830030E0C0001010F0F010100000000000007A
:1003930000000000C030F0C00000000010103070FA
:1003A300D090000000905030107030101010F0F01A
:1003B30010101030701010F0F0101010901070002A
:1003C3000000C06020101010102020F0001010F06A
:1003D300F01010001010F0F01010008080FFFF806C
:1003E30080808040603F1F008080FFFF808000F09E
:1003F3006143838686CC7C38008080FFFF8484043D
:10040300060301008080FFFF8080808080C03080F1
:10041300C0E09C0B0808098FFEF0C08000000000BC
:100423008183FEFC82810000000000008080FFFFCA
:1004330080800000008080FFFF8282828F80C02046
:10044300001F3F60C080808080804020008080FF4C
:0B045300FF8282028282FFFF80800097
:00000001FF
